:020000040000FA
:0600000002EF0CF01200FB
:0600080004EF04F01200F9
:060018000CEF04F01200E1
:0608000002EF0CF01200F3
:0608080070EF09F0120080
:0608180072EF09F012006E
:06082A000100301800007F
:08083000970000000700000022
:08083800F6EC08F06A6A686A38
:100840009F0E6B6EFB0E696E6D8C6D9C6E6ADAECA2
:1008500008F0DF6ADF50006E016A060E005C000ED1
:10086000015810E2DF50040DF3CFE9FFF4CFEAFFA7
:10087000000EE926040EEA22EE6AEE6AEE6AEE6ADD
:10088000DF2AE8D7160E706E68A604D0030EA6EC19
:1008900008F0FAD70001776B7C6B7D6B7E6B6D98EF
:1008A000040E6D6F040E6E6F616B606BF9EF08F0F4
:1008B000F6EC08F0000160510BE16D6A696A6DB6F3
:1008C00002D06D86FCD70001010E606F140E6F6EB2
:1008D000600508E16DBA06D0686A696A698069884E
:1008E000020E606F6850040B04E06950040B01E0D5
:1008F00069D86DB24CD06850010B11E06950010B02
:100900000EE09ADF0001040E606F0401180E026F02
:10091000040E036F080E016F006B8C0E00136850FD
:10092000100B07E06950100B04E046D8040EA6EC4B
:1009300008F06850400B08E06950400B05E0F2EC0D
:1009400009F0060EA6EC08F06850200B04E0695090
:10095000200B01E01ED86850020B06E06950020B24
:1009600003E0F3EC09F06A6A040E0001605D0FE336
:1009700069A60DD0DF6A040EDF5C09E268A607D025
:100980006CCF84F0030EE2DB27D8DF2AF4D7F9EF2F
:1009900008F070A00ED0CDEC08F0EF50800808E110
:1009A000DFDBEF50840804E1CDEC08F08C0EEF6E35
:1009B0007090050EA6EF08F06984040EC7DB6D8207
:1009C000F0EF09F06D92F1EC09F0699468A403D09E
:1009D000020EBCDBFBD71200FD0E0001841518E1EE
:1009E0007E0E8415E8407F0B040DF3CF63F0F4CF47
:1009F00064F0000E6327040E642363C065F064C0D6
:100A000066F04AEC09F002E10EEF05F01FEF05F089
:100A1000FD0E8415040801E11AD81200A1DBEF5085
:100A2000800B02E09DDBEF6A0001736B746B786BE7
:100A3000796B776B93D8F4EC09F0D2EF06F0020EE5
:100A40000001745D02E15CEF07F052EF05F0CEDBD0
:100A500087DBEF50400B01E0010EDF6E080E000156
:100A6000605D09E11AC46EFF6E50000802E2100ECC
:100A700001D0040E606F740513E13CEC09F0CAD993
:100A8000020E0001735D03E16BDB840E07D0DF50C3
:100A900003E166DBC80E02D063DB880EEF6E01D087
:100AA00001D8A7D3E4DB030EE126020E0001745D3A
:100AB0002BE16D50100B28E070DBEE52EF50006E12
:100AC000016A080E001820E101501EE1E3DB1CE181
:100AD000BDDBEF50800B18E1B9DBBDDBDF6ADF5017
:100AE000006E016A080E005C000E015822E2DF5021
:100AF00088DBDF50EA6A180FE96E040EEA22E5523D
:100B0000E750EF6EDF2AEBD7746BABDBEF6A000EBA
:100B10006D19006E6EC001F0010E00C0DBFF020E09
:100B20006EC0DBFF010EDBCFE9FF020EDBCFEAFF79
:100B3000EF6A00017CAF0CD07F51801107E005D037
:100B400080C0FAFF00017F51F96EFADF00017C9F3F
:100B5000030EE15C02E2E16AE5520BD30401185195
:100B6000600BE842E842E842E842E842000901E05E
:100B7000120019510C0A43E00B0A3FE00C0A31E065
:100B8000010A22E00B0A1EE0020A1CE0030A18E038
:100B9000080A10E0010A0CE00F0A08E0030A01E06D
:100BA00012000001778F080E606F120059EF06F0F7
:100BB000B5EF07F00001610E756F000E766F0CD077
:100BC00094EF06F000EF06F01C510001756F766B94
:100BD000620E7527000E76237781010E786F778F6E
:100BE00012000001778F04011C51EA6A620FE96E5E
:100BF000000EEA221AC4EFFF1200F6EF09F012000D
:100C000036DB040EE12604011A0510E118511F0B12
:100C100000090CE10001778F030E0401195D04E166
:100C20000001010E836F02D00001836B04011A5191
:100C30003AE118511F0B020836E11C510F0B000955
:100C400032E00001778F04011CBF05D0ABDA670EDC
:100C5000E926000E04D0A6DA6D0EE926000ECBDAE6
:100C6000030E195D03E187DA840E1CD01C510F0BB3
:100C7000016A700F006E0F0E0122020E00C0DBFF32
:100C8000030E01C0DBFF020EDBCFE9FF030EDBCF5B
:100C9000EAFFEE90ED521CAF03D06DDA400E02D0A9
:100CA0006ADAC80EEF6E040EE15C02E2E16AE55218
:100CB00060D2800E0401185D36E10001C00E776F2E
:100CC00004011B51030A1EE0010A09E0030A29E19D
:100CD0000001700E756F160E766F120E1FD0A8DA17
:100CE0002A0EF626170E95DA020E0001F76A752510
:100CF000F66E7651F7220900F5CF78F00A00F5CFAD
:100D000079F0120095DA2C0EF626170E82DA75C0ED
:100D1000F6FF76C0F7FF0800F5500001786F796B99
:100D200012000001776B120020DA0401206B216BA6
:100D300018511F0B020A11E0030A0CE0010A22E11C
:100D40000001778F04012081000183051BE104016C
:100D5000208318D00001778F15D00001778F040110
:100D60001CBF05D01FDA670EE926000E04D01ADA80
:100D70006D0EE926000E3FDAFED9EF50040B02E0BB
:100D8000010E206F000177AF07D0200E756F040EA3
:100D9000766F7781020E786F020EE15C02E2E16A03
:100DA000E552E7D16D98000177BF07D07CAF02D044
:100DB00087DA28D056DA840E26D07CBF2AD00401E8
:100DC00018AF23D00001785104011E5D0001795154
:100DD00004011F5904E21EC478F01FC479F01AD828
:100DE0000001010E746FABD9D2D9800EEF6ED5D948
:100DF000EE52080EEF6ED1D92EDACFD9800EEF6EFB
:100E00003BDAAED9C80EEF6E1200000159DAC80EF7
:100E1000EF6E1200AAD90001080E785D000E795914
:100E20000DE278C0DEFF79C0DDFF735102E1010EF3
:100E300003D0730506E1020E736F03D0080EDE6E59
:100E4000DD6A8ED9EF928CD9EF908AD9010EDB50F2
:100E5000EF1286D9EE52DFCFEFFF000EDB50785F46
:100E6000010EDB50795B200E816F040E826F77B12B
:100E70000FD0E5D91BE075C0F6FF76C0F7FF752BE4
:100E8000000E76230800F5509ED9F3E2DB06F1D779
:100E9000D6D90CE075C0E9FF76C0EAFF752B000ECD
:100EA0007623EF5090D9F4E2DB06F2D7020EE15C34
:100EB00002E2E16AE5525DD158D96FD9EE52EFCF27
:100EC000DFFFDFCF00F0005000017D5D000E7E5996
:100ED00003E27DC0DFFF09D0DF50006E016AE850F9
:100EE0007D5D7D6F01507E597E6F010EDB6ADF50A4
:100EF000F36E010EDBCFF4FFF350F45C10E2010E51
:100F0000DB507FD97AC0E9FF7BC0EAFF7A2B000E65
:100F10007B23E552E750EF6E010EDB2AE8D7000E87
:100F2000D8807D55000E7E550CE2C3D936D9EF50DE
:100F3000400B03E18BD9C80E02D088D9880EEF6E22
:100F40000ED084D988D97F51801107E005D080C0A8
:100F5000FAFF00017F51F96EFADF00017C9F020E5B
:100F6000E15C02E2E16AE55204D10001778F22D907
:100F7000010EE66EE66AE66A620EE66E000E91D932
:100F80001AC461F004011A5104E10001100E606FEF
:100F900012000001200E606FF7EF09F0E6D8000E96
:100FA000DE6E040EDD6EFD0EDB50040DF3CF02F09D
:100FB000FE0EDB50080DF3500224006E016A020E93
:100FC0000F0B05E0D89001320032E806FBE1D89023
:100FD00000360136D89000360136D9CFE9FFDACF96
:100FE000EAFF0050EE260150ED22C5D8EF9EFD0E1F
:100FF000DB5002E145D901D048D9EA22DECFEEFF2D
:10100000DDCFEDFFB8D8EF8C020EE15C02E2E16AC1
:10101000E552AFD0AAD8FE0EDB50016A700F006E09
:101020000F0E012200C0DEFF01C0DDFFFD0EDB5010
:10103000E66EA1D8E552E750EE6EED6AFD0EDBA438
:1010400002D0E66AEED8FD0EDBA203D0010EE66EFA
:10105000E8D8020EE15C02E2E16AE5528AD085D866
:10106000FE0EDB5004E1FDD8840EEF6E19D0FD0EAC
:10107000DBCFE6FFFE0EDB50E824E552E724040D4B
:10108000F3CF00F0F4CF01F0000E0026040E012291
:1010900000C0DEFF01C0DDFF840E6DD8E850EF1206
:1010A000020EE15C02E2E16AE55263D05ED8FD0E19
:1010B000DB5002E0EAD801D0E3D89DD85CD8EF7CC1
:1010C0005AD809D9FB0EDBCFEEFFFC0EDBCFEDFFCC
:1010D00052D8EE52FA0EDBCFEFFF400E4CD8E8505C
:1010E000EF16880E48D8E850EF12FD0EDB5002E0F4
:1010F000CCD801D0C5D8EA22DECF00F0DDCF01F098
:1011000000C0F3FF01C0F4FF020EE15C02E2E16AFD
:10111000E5522FD0ACD8010EF36EFC0EDB5004E08C
:10112000D890F336E806FCE1F31C006EFD0EDBCF31
:10113000E9FFFE0EDBCFEAFF0050EF16BDD086D8E8
:10114000EE52080EEF6E82D86BEF09F0E66E680E75
:10115000E66E0F0EE66EDEDFE552E552E552120056
:101160006DC0E9FF6EC0EAFF120081D8020EE126D1
:101170001200E16EA1D0DECFE9FFDDCFEAFF120061
:10118000FE0EEA6ADB34FE0BEA36E96E1200180E38
:10119000EE6E040EED6E26EF09F063C0E9FF64C049
:1011A000EAFF12001C510F0BE96EEA6AD890E9368B
:1011B000EA361200010EE66EE66AE66A710EE66E27
:1011C0000F0E51EF09F0E66E81C0E9FF82C0EAFF21
:1011D000812B000E8223E552E750EF6EDF06010EF1
:1011E0001200200EEE6E040EED6E120040D8E65294
:1011F0001200E55261D0EA22EECFDEFFEDCFDDFF37
:101200001200EA6A200FE96E040EEA22EF50E66E41
:101210001200F7220900F5CF75F00A00F5CF76F03D
:101220001200FE0EDBCFE6FFB9DEE552E5521200FA
:101230001A51F66EF76AD890F636F7361200D9CF03
:10124000E9FFDACFEAFFEE50ED10120065C0E9FFCA
:1012500066C0EAFF12003FD8180EEE6E040EED6E67
:1012600012006DDF94DF8C0EEF6EB0EF08F0D9CF77
:10127000E6FFE1CFD9FF120073DF2DD8F1EF08F0C0
:101280007FDF670EE926000E12007ADF6D0EE92679
:10129000000E120082DFEF503C0BE842E8420D08DE
:1012A0001200E66EE8EC0BF0006E050EE15E0050F9
:1012B000120045DFF1EF08F0E552E7CFD9FF120049
:1012C000020E746F4DDFEE52EF6A4ADFC80EEF6E0A
:1012D000F0DF26EF09F0020EE926000EEA221200E6
:1012E00045D91100D8CFE4FFE0CFE4FFE46E3ED94A
:1012F000E550E5CFE0FFE5CFD8FF1000FC0E8B16E0
:10130000941694848250040B01E0010E00019E6F3C
:1013100012008250040B01E0010E00019E5D07E007
:101320008250040B01E0010E9E6F82A4010C000CA0
:1013300000019C519D1104E1100E9C6F270E9D6FC2
:101340009C07000E9D5B6DA208D09C519D1131E160
:101350008B708B50010B14E129D00001605102E128
:101360008B9024D0600503E18B808B801200020EED
:10137000605D02E18B801AD0040E605D03E18B900A
:101380008B821200100E605D06E100019C519D11E0
:1013900010E18B700BD0200E605D0BE100019C51C1
:1013A0009D1107E18B708B50010B02E08B921200B4
:1013B0008B821200BDDF200E0001605D05E36D50E1
:1013C000020B01E0120056D812000F0EC1121CECE5
:1013D00004F07EEF09F0F9DF58EC04F0EBDFFCD706
:1013E0001200120012001200CBEF0AF012001E0EC3
:1013F000E66E010EE66E0AEC08F0E552E5521200C8
:101400006D840001080EA26F070EA36FA207000EE5
:10141000A35BA251A311FAE16D941200AED80401AE
:101420001B51030A0AE0010A09E11A5107E1DF6AC8
:10143000DF50010803E37FD8FBD71A51E552E5528C
:10144000E7CFD9FF120058EC04F004011B51030A46
:101450000CE0010A06E0030A0CE11A5101E1010C5B
:10146000000C1A5101E1020C000C1A5101E1030CAD
:10147000000C000C82D800019B51740A38E0040A69
:101480001CE0020A53E199519A1102E1000E03D0C7
:101490007BD801E0010E000949E1400EE66E280EFE
:1014A000E66E040EE66EE66A010E58D8F3CF99F0A8
:1014B000F4CF9AF00001700E38D099519A1102E1E0
:1014C000000E03D061D801E0010E00092FE199C0A0
:1014D000E9FF9AC0EAFFEE52EF50000825E2DF5024
:1014E000010802E328D8FBD70001740E1ED09751E3
:1014F000981102E1000E08D097C0E9FF98C0EAFFFA
:10150000EF50800B01E0010E000910E1020EE66EC3
:101510002B0EE66E040EE66E010EE66E1FD8F3CFBC
:1015200097F0F4CF98F00001720E9B6FE552E552F0
:10153000E7CFD9FF1200DF50EA6A280FE96E040EE8
:10154000EA22EF50E66EDF50EA6A2B0FE96E040ED6
:10155000EA22E552E750EF6EDF2A1200E66E56EC03
:1015600008F0006E050EE15E00501200DACFE4FFD5
:10157000E652E552E5CFDAFF1200D9CFE6FFE1CF20
:10158000D9FFE652DF6A120099C0E9FF9AC0EAFF6C
:06159000EF50800B120079
:0A159600040118511F0B010801E0C9
:1015A00012001C5101E01200060E195D21E11B51D1
:1015B000230A1BE0010A0CE0030A1AE1000161059D
:1015C00017E10001940E756F160E766F090E09D0A3
:1015D000000161050DE10001FB0E756F160E766FBF
:1015E0002F0E786F796BC00E02D00001800E776FDE
:1015F00004011851600BE842E842E842E842E84240
:10160000010801E0120019510B0A2AE0080A1DE046
:10161000090A15E0080A09E00B0A05E0080A01E0DA
:10162000120036EF0BF037EF0BF00001A40E756FD0
:10163000000E766F010E786F796BC10E0FD000012E
:10164000800E776F1BC4A4F012000001A50E756F09
:10165000000E766F010E786F796B810E776F120036
:101660000001800E776F1AC4A5F01200120012005C
:10167000120110010000000825090170010001029B
:10168000000109022900010100C032090400000222
:1016900003000000092111010001222F000705812C
:1016A00003080001070501030800010403090434CD
:1016B000034D006900630072006F006300680069F9
:1016C000007000200054006500630068006E006F29
:1016D000006C006F0067007900200049006E006315
:1016E000002E001803470065006E00650072006957
:1016F000006300200048004900440006A0FF0901E3
:10170000A1010903150026FF007508950281020951
:1017100004150026FF0075089502910209051500C1
:1017200026FF0075089502B102C08216AB16AF16EF
:02173000E316BE
:0E1732002A0EF66E080EF76E000EF86E00011D
:101740000900F550926F0900F550936F03E192671D
:1017500001D03DD00900F5508D6F0900F5508E6F16
:101760000900F5508F6F09000900F550E96E090076
:10177000F550EA6E090009000900F550906F090064
:10178000F550916F09000900F6CF94F0F7CF95F06E
:10179000F8CF96F08DC0F6FF8EC0F7FF8FC0F8FF30
:1017A0000001905302E1915307E00900F550EE6EFD
:1017B0009007F8E29107F9D794C0F6FF95C0F7FFBC
:1017C00096C0F8FF00019207000E935BBFD712008E
:1017D000FE0EE3CFE9FFFF0EE3CFEAFFE9CFF3FF11
:1017E000EACFF4FFFB0EE35003E1FC0EE35009E007
:1017F000FB0EE30602E2FC0EE306FD0EE350EE6E86
:04180000F1D712000A
:0C18040013EE00F023EE00F0F86A049CE4
:1018100099EC0BF017EC0CF0EBEC09F0FBD7120095
:0E18200000EE00F00F0EEE6AEA62FDD7120035
:02182E001200A6
:07183000000000007200003F
:00000001FF
